:04000000830113283D
:10000800FD00030EFE0083010A08FF008A11722F0B
:100018007F088A007E0E8300FD0E7D0E09001720E2
:10002800EF30FC00542A213084001C20A0308400CA
:100038005030A0008001840AA00B1E280800F90097
:10004800A2208A01F4004D208A01F5004D208A0182
:10005800FA0003107A08FB00703084004D208A01F2
:100068000006031D0314840AFB0B3228031C4628D0
:1000780054205420FF30F407031CF503740875045A
:10008800031D2D284D208A01FB004D208A007B0886
:100098008200F90FF803F80A78088A0079088200C4
:1000A800F90FF803F80A08007C07F000F1010800CE
:1000B8007C078400831308007108F5007008F400B9
:1000C800080002307407840072088000840A7308EC
:1000D80080006E28740A84007108800074087528EE
:1000E80074088400700880000800F11B7D287008DF
:1000F800FF298B209628F11B83287008072A8B205C
:100108009828F11B89287008FB298B2090287108F2
:10011800F800F81370080800F900A2208A01F0001E
:10012800F008080098209B28F900703084009C2073
:10013800A2208A018000840AF90A080078088A0047
:10014800790882000530030503190800053C0800FA
:100158007108750680397130031DBC28AC297008F8
:10016800740680397030031DBC287408F00208003A
:100178008400801F0314801B031008007C07840080
:1001880083130008F00008007C0784008313082A02
:100198007C07840083130822002A7C0784008313C9
:1001A8000008F40008007C0784008313212AF10169
:1001B800F01BF1030800F101F01BF1037108E528B9
:1001C8000030F11BFF30F200F3000800F501F41BCA
:1001D800F5030800F501F41BF5037508F428003051
:1001E800F51BFF30F600F7000800F101F201F301FA
:1001F80008000121182904211829FB1388211F2927
:100208008F211F290A2116290D211629FB138A215E
:100218001F2992211F291B2112291E212708F300BB
:100228002608F2002508F1002408F0000800FB1356
:100238009D211F299421A401A501A601A70103104E
:10024800A00DA10DA20DA30DA40DA50DA60DA70D22
:1002580077082702031D3A2976082602031D3A2942
:1002680075082502031D3A2974082402031C4B292A
:100278007408A402031C52217508A502031C562108
:100288007608A602031CA7037708A7020314F00D3B
:10029800F10DF20DF30DF90B23298529FF30A50780
:1002A80003180800FF30A60703180800A703080072
:1002B800FB1388216A298F216A29FB138A216A295D
:1002C80092216A29FB139D216A299421741C7A2999
:1002D8002008F0070318C7212108F1070318C921CE
:1002E8002208F2070318F30A2308F307A00DA10D4B
:1002F800A20DA30D2010F70CF60CF50CF40CF90B5D
:100308006A29FB1F0800BB29F101F501F201F6017A
:10031800F301F7019D29DF20EE209429E420F32042
:10032800FB13730877068039FB04F31BBB21F71B0B
:10033800C0212030F9007008A0007108A1007208DF
:10034800A2007308A300F001F101F201F301080013
:1003580075087102031D08007408F0020800C22124
:100368007408F0070318F10A7508F1070800F30983
:10037800F209F109F009C529F709F609F509F4099F
:10038800CD29F00F0800F10F0800F20F0800F30A5A
:100398000800F40F0800F50F0800F60F0800F70A28
:1003A8000800F400F821031908000310F00DF10DFE
:1003B800F40BD9290800F400F40803190800031005
:1003C800F00DF40BE3290800F400EC29F917F11FEC
:1003D800F913F821031908000310F91B0314F10C91
:1003E800F00CF40BF0290800740875040800840068
:1003F8000008F00008000722840A0008F200840AB6
:100408000008F300080084000008F000840A0008CF
:10041800F10008007C0AFC0AFC0AFC0AFC0A8313A7
:100428002022840A0008F600840A0008F700080061
:100438007C0AFC0AFC0A831384000008F400840A7E
:100448000008F500080083137C0884007308800006
:10045800840372088000FE30FC0783137C08840044
:1004680071088000FC03392AF00083137C0884009B
:1004780070088000FC03080083137C08840075085A
:100488008000FC0383137C08840074088000FC034C
:1004980008008313FC0A7C0884000008F4000800A4
:1004A800552AF430FC076430F000F10131228A1536
:1004B800B2240230FC078A11C925871085128A11D7
:1004C800D8268A11BC278A156F238A15B020F630E2
:1004D800F0008F30F10031228A15E8200230FC0745
:1004E8000130F000F1013122F001F10131228A15C9
:1004F80097200430FC07ED30F0008F30F1003122F6
:100508008A15E8200230FC07E830F0000330F100DB
:1005180031228A15B2240230FC078A15B0208A11CC
:1005280007260C305C20700880000C305C200030FE
:1005380000028A110319C72A8A010130F000F1016B
:1005480031228A15B2240230FC078A1107260C30A2
:10055800D120740870028A11031DC72A8A010C3041
:100568005C20013000028A11031DBD2A8A018A110C
:10057800BE240C305C20023000028A11031DC72AF9
:100588008A018A11BE240B0880388B000B0820389A
:100598008B000B0810388B0007305C20013080007E
:1005A800840A80010130F00039220830C820312245
:1005B8008A1121270330FC070A305C208001ED01F5
:1005C8000B305C2001308000EB01EC0109305C202D
:1005D8000230800003305C2000308000840A8001F3
:1005E8008316093021028312A6208A1103194D2B84
:1005F8008A018316A1018312ED0A3D306D028A112A
:10060800031D092B8A010130ED0083136B3007228B
:10061800FF30F400F501AC21A6208A110319182B2C
:100628008A01FF30EB00EC016D08F000F1012E307B
:10063800F400F501B421700883137118831784003E
:100648006B0880000330C820312283136B300722E7
:1006580039228A15CD230330FC0703305C20013092
:100668008007840A0318800A0330C820FF30F4008A
:100678001F30F500AC21A6208A1103194B2B8A01E3
:1006880003305C20FF308000840A1F308000EB01BB
:10069800EC0105305C2000308000840A80016D0880
:1006A800643EAC000B30C2200630F4005C217008B8
:1006B800AD00AB012D082B028A1103188D2B8A017E
:1006C8002B082C02AA0064302A02A6208A110319DA
:1006D800732B8A012A089C3EAA008A11762B2A08C5
:1006E800D83EAA002A08F000F1012E30F400F501E6
:1006F800B42185206220F5010530C820B4210530D9
:100708005C2070088000840A71088000AB0A8A1196
:100718005E2B01306E028A11031D962B8A018A1105
:10072800FC26EE018A1107260C305C207008800038
:100738000C305C20003000028A110319E32B8A0177
:100748000130F000F10131228A15B2240230FC0791
:100758008A1107260C30D120740870028A11031DF3
:10076800E32B8A010C305C20013000028A11031D42
:10077800CD2B8A010B305C20800A0B305C200B30BB
:1007880000028A11031DCD2B8A010B305C20013039
:1007980080000C305C20023000028A11031DE32B1C
:1007A8008A010A305C20800A0A305C20033000028B
:1007B8008A11031DE32B8A010A305C2080010A306C
:1007C8005C20003000028A11031DF82B8A010130D9
:1007D800F000F1013122F001F10131228A15972050
:1007E8000430FC078A1188260A305C200130000298
:1007F8008A11031D562C8A010130F000F1013122C3
:10080800F001F10131228A1597200430FC070B30E2
:10081800D120F5010530C8200A217C0A8400831301
:1008280070088000840A710880000930C220F10134
:1008380060200130582031227F20B3211C226E20F5
:100848007C0AC920F401F501AC208A110318342C64
:100858008A017C0A8400831300308000840A8001A6
:100868007C0AC9200A30F400F50164217C0A84005E
:10087800831370088000840A710880000430F00037
:1008880039220230C820E42027228A1509210530A0
:10089800FC07E830F0008F30F10031228A15E8209B
:1008A8000230FC070A305C20023000028A11031D66
:1008B8008A2C8A01F00139228A151C22FC0A7C0A3A
:1008C8008400831370088000840A71088000013056
:1008D800F000F1013122F001F10131228A1597204F
:1008E8000430FC070430F00039220230C820E4202C
:1008F80027228A1509210530FC07E330F0008F30E4
:10090800F10031228A15E8200230FC07F001F101DC
:100918003122F001F10131228A1597200430FC07B9
:100928000430F00039220630C820FA2027228A1520
:1009380009210530FC07E130F0008F30F100312249
:100948008A15E8200230FC070230F00039220C300A
:10095800C220F92027228A1509210530FC07DF303B
:10096800F0008F30F10031228A15E8200230FC07B0
:100978008A11F42AFE30FC0785168A15B020F0018A
:10098800F1013122F001F10131228A15972004305A
:10099800FC07D730F0008F30F10031228A15E820AB
:1009A8000230FC070130F000F1013122F001F101C1
:1009B80031228A1597200430FC07CE30F0008F30A2
:1009C800F10031228A15E8200230FC07BD30F00022
:1009D8008F30F10031228A15D2220230FC076430B0
:1009E800F000F10131228A15B2240230FC07AA3046
:1009F800F0008F30F10031228A15D2220230FC0734
:100A08006430F000F10131228A15B2240230FC076B
:100A18009B30F0008F30F10031228A15D22202304B
:100A2800FC076430F000F10131228A15B22402304B
:100A3800FC078B30F0008F30F10031228A15D2226A
:100A48000230FC078630F0008F30F10031228A1521
:100A5800D2220230FC078130F0008F30F1003122C1
:100A68008A15D2220230FC0702305C2080018A15E8
:100A7800262402305C20700880000230C2200F302B
:100A8800F8004F3023288A1172258A116D2D7C3089
:100A9800F0008F30F10031228A15D2220230FC0793
:100AA8008A116D2D7730F0008F30F10031228A15D0
:100AB800D2220230FC078A116D2D6030F0008F3091
:100AC800F10031228A15D2220230FC0785128A11E0
:100AD8006D2D8A111D2D0230FC070800FE30FC0721
:100AE8004130F0008F30F10031228A15D2220230D5
:100AF800FC077C0A8400831300308000840A80018C
:100B08007C0AC920E830F4000330F500AC218A11D2
:100B18000318C62D8A010430F00039220230C8209B
:100B2800FA2027228A15ED220530FC073F30F00015
:100B38008F30F10031228A15D2220230FC070330AF
:100B4800F00039220230C82031228A15772302307A
:100B5800FC07F92027228A15ED220530FC073D30D5
:100B6800F0008F30F10031228A15D2220230FC07C2
:100B78007C0A8400831301308007840A0318800AE2
:100B88008A11842D0230FC0708008316173085006F
:100B980083128316013086008312831689308700FA
:100BA800831285018316C7308100831281018F016A
:100BB8008E010730900080309F0083160E309F0012
:100BC80083120C3097000130F0003922F001F10156
:100BD80031228A1121270330FC078316FF30920047
:100BE80083127F3092008B0108007C0A84008313F3
:100BF8000008AA002A088A110319062E8A018A11F8
:100C0800AA0B032E080003018518013E003E8A1135
:100C1800031D132E8A010130AA008A11202E030118
:100C28000519013E003E8A11031D1F2E8A0102305C
:100C3800AA008A11202EAA012A08F0000800FC0345
:100C48008A1107267C0A84008313700880006430A8
:100C5800F000F10131228A15B2240230FC078A1112
:100C680007267C0AD220740870028A11031D472EB9
:100C78008A010A30F000F10131228A15B2240230CB
:100C8800FC078A11332E0A30F000F10131228A154F
:100C9800B2240230FC077C0AC320FC0A0800083092
:100CA8006F028A11031D5D2E8A018316A00A831222
:100CB800EF0183163C30200283128A11031D6B2E2C
:100CC8008A018316A20A83128316A001831283164F
:100CD8003C30220283128A11031D792E8A01831661
:100CE800A30A83128316A201831283160D302302EE
:100CF80083128A11031D872E8A018316A40A831280
:100D08008316A30183120800FE30FC07831623080C
:100D18008312F000F1017C0A8400831370088000BC
:100D2800840A710880007C0AC920FA2027228A15C3
:100D3800C8210430FC073A30F00039228A15DA203D
:100D4800FC0A831622088312F000F1017C0A840051
:100D5800831370088000840A710880007C0AC92007
:100D6800FA2027228A15C8210430FC073A30F000FF
:100D780039228A15DA20FC0A831620088312F0002B
:100D8800F1017C0A8400831370088000840A7108CA
:100D980080007C0AC920FA2027228A15C82104303D
:100DA800FC070230FC0708008316A401831283168F
:100DB800A30183128316A20183128316A001831252
:100DC800EF010800F00139228A151C22FC0A70087C
:100DD800AA007108AB000330F000392283132A30CF
:100DE8000722FA2027228A1509210530FC07080066
:100DF80087140530F00039228A11F925FC0A87107A
:100E08000530F00039228A11F925FC0A87140530CB
:100E1800F00039228A11F925FC0A87100530F00004
:100E280039228A11F925FC0A87140530F000392285
:100E38008A11F925FC0A871008007C0A84008313AC
:100E48000008AA00840A0008AB002A30F000F1016B
:100E580031227F200230F400F501EC211C226E20A3
:100E680083132A3007220030F1057008AC000330E4
:100E78005C20013000028A11031D472F8A012C08CB
:100E880095008A11492F2C089B007C0A8400831343
:100E98000008AA00840A0008AB002A30F000F1011B
:100EA80031227F200430F400F501D6211C226E2067
:100EB80083132A3007220C30F0047008AC0003308A
:100EC8005C20013000028A11031D6F2F8A012C0853
:100ED80097008A11712F2C089D0008008A110B1D9C
:100EE800B02F8A01FB308B05EF0A08306F028A1198
:100EF800031D862F8A018316A00A8312EF01831629
:100F0800A10A831283163C30200283128A11031D22
:100F1800942F8A018316A20A83128316A0018312D2
:100F280083163C30220283128A11031DA22F8A01E4
:100F38008316A30A83128316A201831283160D3027
:100F4800230283128A11031DB02F8A018316A40A73
:100F580083128316A30183128A118B1CBB2F8A016B
:100F6800FD308B050130EE00EC0AEB0FEC030C288A
:100F78006430F000F10131228A15B2240230FC07F6
:100F8800F001F10131222330F000F10131228A15FC
:100F980024200430FC07F001F10131222330F00055
:100FA800F10131228A1524200430FC07F001F101F7
:100FB80031222330F000F10131228A152420043037
:100FC800FC07F001F10131222230F000F101312259
:100FD8008A1524200430FC07F001F1013122283061
:100FE800F000F10131228A1524200430FC07F001B9
:100FF800F10131220C30F000F10131228A15242050
:101008000430FC07F001F10131220630F000F10153
:1010180031228A1524200430FC07F001F101312225
:10102800F001F10131228A1597200430FC070A30BB
:10103800F000F10131228A15B2240230FC070800C1
:101048008A017C0A840083130008AA00840A000825
:10105800AB0006080F39382283132A300722F030F4
:10106800F0050030F1054D22F50140221C22B42183
:101078007008AA007108AB002A0886000330C8204F
:101088000130F400F501AC208A15031D50288A01AF
:10109800083086048A1553288A01F73086058A01A4
:1010A80004308604FB3086057C0A8400831300081C
:1010B800AA00840A0008AB002A30F000F1013122AE
:1010C8007F200430F400F501D6211C226E2006088A
:1010D8000F39382283132A300722F030F005003008
:1010E800F1054D22F50140221C22B4217008AA0006
:1010F8007108AB002A0886000330C8200130F400CC
:10110800F501AC208A15031D8E288A010830860453
:101118008A1591288A01F73086058A0104308604E9
:10112800FB30860508008A01F001F1013122053003
:10113800C8200630F400F501D62131220530C82038
:101148008030F0070318F10A1C22B42131228A15D5
:1011580024200430FC0708008A01F001F101312243
:101168000130F000F10131228A1524200430FC07F7
:101178000230F000F10131228A15B2240230FC0756
:1011880008008A01F001F10131220230F000F1017A
:1011980031228A1524200430FC070230F000F101C6
:1011A80031228A15B2240230FC0708008A01013076
:1011B800F000F10131220330C220DB2031228A15F0
:1011C80024200430FC0708008A017C0AC9208520F5
:1011D8008A15031907298A010130F000F10131222B
:1011E8000330C8208520F10131228A1524200430DB
:1011F800FC077C0A8400831301308007840A0318E3
:10120800800A8A15E8288A0108008A01F630FC0756
:101218000F305C2080037C0A840083130030800038
:10122800840A80018A017C0AC9200830F400F5018B
:10123800AC208A15031851298A018A010B30CC2069
:101248000A30F400F501F601F70111217C0AD820D3
:10125800272207305820B4210E2246224D2270083A
:101268008313711883178400740880000B3058208A
:10127800312279200A30F400F501F601F7011E2128
:101288001C2265208A017C0A8400831301308007B0
:10129800840A0318800A8A1516298A010F30C22089
:1012A800F1017C0A8400831370088000840A7108A5
:1012B80080008A017C0AC920F401F501AC20A6202F
:1012C8008A1503197F298A018A017C0AD8200330EC
:1012D8005820B4218520303E38228A15DA20FC0AAD
:1012E8008A017C0A8400831301308002840A031C6B
:1012F80080038A155D298A01033058208520303EF5
:1013080038228A15DA20FC0A0A30FC0708008A010C
:10131800FC030230C2200A30F400042102305C20B1
:10132800700880007C0A8400831380018A017C0A8B
:10133800C3200A30F400B3208A150318C5298A018E
:101348008A017C0AD2200230C220B320A6208A1546
:101358000319B7298A01FF30F00039228A15DA20EB
:10136800FC0A8A15BE298A015F30F00039228A15E5
:10137800DA20FC0A8A017C0A84008313800A8A1511
:101388009A298A01FC0A08008A01FE30FC07AA0192
:10139800AB018A0183132A3007220230F400F501D9
:1013A800AC208A150318052A8A018A010330CC204B
:1013B8000A30F400F501F601F701112183132A30F0
:1013C8002022272205305820B4210E2246224D2201
:1013D8007008831371188317840074088000033021
:1013E8005820312279200A30F400F501F601F7017E
:1013F8001E211C2265208A01AB0AAA0FAB038A159D
:10140800CD298A0101305820F10AF00FF103852017
:10141800303E38228A15DA20FC0A0130582085200F
:10142800303E38228A15DA20FC0A0230FC07080010
:101438008A01FC037C0A84008313800183168030B0
:101448009F04831202305820312285200330F40093
:10145800E0211C22742002305C20383080050230E4
:101468005C204130800402305C2000089F0001307D
:10147800F00039228A11F925FC0A04309F048A01F8
:101488007C0AC3208A150319572A8A011F080439C0
:10149800F0007C0A84008313700880007C0A8400B2
:1014A80083138A15432A8A011E08F000F101700887
:1014B800AC007108AD0083132C3007220830F4000B
:1014C800F501D6217008AA007108AB0083161E0822
:1014D8008312F000F1017008AC007108AD008313AD
:1014E8002C30202283132A300722B4217008AA0046
:1014F8007108AB0040309F0083132A300722FC0A92
:1015080008008A017C0A84008313000803178D00F1
:1015180003130317831601308C0003138312031778
:101528000C080313AA002A08F00008008A017C0AA4
:1015380084008313000803178D00031302305C2016
:10154800000803178C000313031783168B138C13DF
:101558000C1555308D00AA308D008C140C1180307C
:101568008B040130AA008A0100302A028A15031967
:10157800C72A8A01031783160C080313831202393A
:10158800AA008A15B72A8A01031783160C080313C1
:1015980083120839AA002A08F00008008A017C0A88
:1015A800C92085208A150319EB2A8A017C0AC920DB
:1015B800852039228A154024FC0A7C0A840083137A
:1015C80001308007840A0318800A8A15D22A8A0102
:1015D80008008A01F630FC070F305C2080037C0A83
:1015E8008400831300308000840A80018A017C0A09
:1015F800C9200830F400F501AC208A150318352BF2
:101608008A018A010B30CC200A30F400F501F6017A
:10161800F70111217C0AD820272207305820B4214D
:101628000E2246224D2270088313711883178400F6
:10163800740880000B305820312279200A30F400D9
:10164800F501F601F7011E211C2265208A017C0A9A
:101658008400831301308007840A0318800A8A15DE
:10166800FA2A8A010F30C220F1017C0A8400831310
:1016780070088000840A710880008A017C0AC920E9
:10168800F401F501AC20A6208A150319632B8A0101
:101698008A017C0AD82003305820B4218520303EA6
:1016A80038228A154024FC0A8A017C0A84008313A4
:1016B80001308002840A031C80038A15412B8A01A9
:1016C800033058208520303E38228A154024FC0AF1
:1016D8000A30FC0708008A010230F00039228A1516
:1016E8005B24FC0A08008A017C0A84008313000832
:1016F800AA00840A0008AB0083132A3007220030AE
:10170800F10570088316A500831283132A30072277
:101718000830F400F501EC2170088316A600831246
:101728008A15A5240530F0003922A030F0003922AE
:101738008A1563240230FC070430F000392283162E
:101748002608831238228A1563240230FC070430E5
:10175800F000392283162508831238228A1563245B
:101768000230FC07103087040530F0003922A13020
:10177800F00039228A1563240230FC0783160830EA
:10178800870483120430F00039228A155B24FC0A8E
:1017980008008A0102305C200008AA00840A0008B8
:1017A800AB0083132A3007220030F1057008831636
:1017B800A500831283132A3007220830F400F501AC
:1017C800EC2170088316A60083127C0A8400831318
:1017D80000088316A70083128A15A5240530F00097
:1017E8003922A030F00039228A1563240230FC0720
:1017F8000430F000392283162608831238228A150D
:1018080063240230FC070430F000392283162508CF
:10181800831238228A1563240230FC070630F00050
:10182800392283162708831238228A156324023046
:10183800FC070530F000F10131228A15B22402308C
:10184800FC070800871B262C0830F9008A150A12A5
:101858000530CA248A150A120C30C8240310871BC5
:101868000314F00C8A150A12F90B2E2C8A150A1289
:10187800871F3C2C8A0108008A017C0A8400831394
:1018880003100930FB0003180717031C07138A15F8
:101898000A120C30C824800C8A150A12FB0B472C3C
:1018A80007178A150A120F30C8248A0108008A010E
:1018B8007C0A84008313083000048A156B2C8A0183
:1018C8007C0A840083130008F000840A0008F400EE
:1018D8008A15741C702C8711073084000830F100B9
:1018E80000128A15F419832C8A158011F00D03183B
:1018F800801500160012F10B792C8A158D2CF00139
:1019080003108A15001680190314F00D0012F10B4C
:10191800862C801184178015741980118413001681
:101928008019F10A00128015841780118413710838
:10193800F41DF0008A01F41C0800801100168015BF
:101948000800073084000830F1008A1500160012DC
:10195800F10BAA2C0230F4008A158E2C8A017C0A1D
:10196800C9208A150A12700871040319C62C8A1531
:101978000A12A930C8248A150A12F003700FB72C6E
:10198800F103B72C8A01080000000000F400F40BF2
:10199800CB2C0800F500F030CA24F50BCF2C08003A
:101E7A000A3400342C340034743469346D346534D3
:101E8A002C34203463346F3475346E347434203413
:101E9A000A3400340434003401343134473405340C
:101EAA0032344B34053433345634053465346134B2
:101EBA0005346D34053445346E34643420346F345B
:101ECA006634203450344334203463346F346E34EF
:101EDA006E3465346334743469346F346E34203448
:101EEA000A3400342034333420340A3400342034A1
:101EFA00323420340A34003433343A3420340A3445
:101F0A00003432343A3420340A34003431343A3426
:101F1A00443475346D347034203445344534503487
:101F2A0052344F344D3420340A3400345334653437
:101F3A007434743469346E34673420344D346534FF
:101F4A006E34753420340A34003447344D34203426
:101F5A0043346F3475346E347434653472342034D7
:101F6A005634653472342E34353420340A3400340D
:101F7A002034533474346134723474342034503419
:101F8A0072346F346734723461346D3420340A34F5
:101F9A00003447344D343C342D343E3450344334C9
:101FAA00203400344D3465346E3475342034203492
:101FBA00203400346D3400342F3400344234613418
:101FCA00743474340034753453342F346834003420
:101FDA00303431342F34303437342F3430343134D0
:101FEA00003454344534533454342034563445344C
:041FFA005234003429
:00000001FF
